:1017000039C057C083C055C054C053C052C051C027
:1017100050C04FC04EC04DC04CC04BC04AC0040367
:10172000090422036300720065006100740069000F
:101730007600650070006F006E0079002E00630077
:101740006F006D000C03750042006F006F007400A5
:1017500012011001FF000008C016DC0501010102A2
:10176000000109021200010100803209040000009A
:101770000000000011241FBECFE5D2E0DEBFCDBFC8
:1017800000EB0F9307E00F9310E0A0E6B0E0EAEF64
:10179000FFE102C005900D92A636B107D9F710E01F
:1017A000A6E6B0E001C01D92AB39B107E1F7EED17A
:1017B00022C4A6CFA82FB92F80E090E041E050EAE4
:1017C000609530E009C02D9182279795879510F09C
:1017D00084279527305EC8F36F5FA8F30895EADF8A
:1017E0008D939D930895A6E088279927AA9569F07F
:1017F0000197E1F3B399FCCFB39BFECF81E099272A
:10180000A6B3019611F0A871D9F70895CF93CFB779
:10181000CF93C0915F02C03B21F4C0915E02C730FC
:1018200021F0CF91CFBFCF916ACFCC27C395B39B87
:10183000E9F7B39B0BC0B39B09C0B39B07C0B39B35
:1018400005C0B39B03C0B39B01C0D3C00F92DF930D
:10185000C0917E00DD27CB57DF4F012EB39B03C025
:10186000DF910F90E6CF2F930F931F934F932FEF9E
:101870004F6F06B303FB20F95F933F9350E03BE0CB
:1018800065C016B30126502953FDC89556B30127EC
:1018900003FB25F92F7306B3B1F05027102713FB74
:1018A00026F906B22230F0F000C016B3012703FB80
:1018B00027F90126502906B22430E8F54F77206831
:1018C00016B30000F6CF50274F7D206206B2102FCE
:1018D000000000C006B300265029102713FB26F98C
:1018E00006B2E2CF4F7B06B3206400C0DACF0126F8
:1018F0005029187106B269F14E7F2160012F16B38D
:1019000028C0002650294D7F06B22260102F29C022
:10191000012650294B7F06B22460012F2DC016B33B
:1019200001265029477F2860000006B22EC04F7E56
:1019300006B3206130C0422706B3499300265029E0
:10194000102706B24FEF13FB20F9297F16B379F267
:10195000187159F10126502906B2012703FB21F91C
:10196000237F06B371F2002650293150D0F006B221
:10197000102713FB22F9277E16B351F201265029B6
:10198000012703FB06B223F92F7C49F2000006B3BE
:10199000102713FB24F90026502906B22F7939F2BB
:1019A00070CF10E21ABF002717C03B503195C31B00
:1019B000D04010E21ABF0881033CF9F00B34E9F083
:1019C00020917C001981110F1213EDCF093651F1CE
:1019D0000D3211F0013E39F7009383003F915F9182
:1019E0004F911F910F912F91DF910F90CAB7C5FDB5
:1019F0001DCFCF91CFBFCF91189520918300222387
:101A000069F310918100112321F5343022F13093D4
:101A1000810020937D0010917E003BE0311B3093CC
:101A20007E0019C00091810001309CF40AE53091DC
:101A3000600034FD11C000936000C1E7D0E010C029
:101A4000052710E000C021C0052710E0C89508BB9D
:101A500014C03AE501C032ED032EC0E0D0E032E020
:101A600017B31861C39A08B317BB58E120E84FEFCA
:101A700020FF052708BB279517951C3F28F7000076
:101A80004552B0F720FF0527279508BB17951C3F47
:101A9000B8F629913A9561F7077E10918200110FEF
:101AA00008BBC250D04011F010937C0010E21ABF66
:101AB000086017B3177E402F477E54E05A95F1F720
:101AC00008BB17BB48BB8ACF81E080936D00F894B8
:101AD000E0916700F0916800329785E080935700AD
:101AE000E89507B600FCFDCF789408952091670033
:101AF000309168002115310589F124303105B1F0AC
:101B000046E12C3F340739F48091690090916A00D6
:101B10008E579B4F0DC046E12E3F340749F480910C
:101B20006B0090916C008D579B4F02C08FE79BEC30
:101B3000F894E0916700F091680021E00C01209397
:101B40005700E8951124789480916700909168007F
:101B500002969093680080936700089581E18093D6
:101B60005700E895E3CFCF93DF93C0916700D09102
:101B70006800CF73D0708FEF9FEFB8DF2296C0342C
:101B8000D105CCF3A1DFDF91CF910895DF93CF93FF
:101B90000F92CDB7DEB788E10FB6F89481BD11BCC6
:101BA0000FBEE0E0F0E0859194912BEC8F37920727
:101BB00041F4E4E0F0E0859194913BEC8F3793079A
:101BC00009F0D1DF1092680010926700AC9A8BB7D1
:101BD00080628BBFBB9A8FE49DE2A9E18150904067
:101BE000A040E1F700C00000BB987894EE24FF24E9
:101BF00020918100235027FDF3C080917E00ECE00E
:101C0000F0E0E81BF109EB57FF4F80917D008D322A
:101C100009F0A3C0283009F0E1C083EC8093710083
:101C20008AE58093600010926E002081922F90765A
:101C30008181992321F1882341F482E690E09093F9
:101C4000800080937F0024E07EC0813069F482812F
:101C500080936F00848195819093680080936700E2
:101C600027FD6CC02FEF6BC090916600823011F49D
:101C7000916001C094609093660020E064C09281FE
:101C800010927A00882331F410927B008AE790E06A
:101C900022E04FC0853019F49093820040C0863016
:101CA000A9F58381813019F480E597E104C0823081
:101CB00041F482E697E19093800080937F0022E1D7
:101CC00021C08330F1F4992341F48EE197E19093A0
:101CD000800080937F0024E015C0913041F482E2BF
:101CE00097E19093800080937F0022E20BC09230B6
:101CF00041F484E497E19093800080937F002CE08E
:101D000001C020E080E480936E001DC0883059F04F
:101D1000893019F49093840002C08A3039F08AE740
:101D200090E020E006C084E890E002C08AE790E0FE
:101D300021E09093800080937F0005C0268180E899
:101D400080936E0007C08781882321F486818217E3
:101D500008F4282F2093610041C080916E0087FF16
:101D60003DC080916F00821B80936F008F01809136
:101D7000670090916800009749F4D8018D919C917B
:101D8000119790936A008093690014C08430910584
:101D900041F4F8018081918190936C0080936B00F5
:101DA00009C0F6E18A3F9F0728F081E18093570040
:101DB000E89509C0D8018D919D918D01298396DE0A
:101DC00029812250A1F680916F00882339F48091F7
:101DD000660082608093660010926100109281001C
:101DE0008091600084FF47C0809161008F3F09F4BB
:101DF00042C0082F893008F008E0801B8093610002
:101E00008091710098E8892780937100002339F14F
:101E1000E0917F00F091800090916E00802F8150C2
:101E200096FF0CC090E08D589F4FA2E7B0E0249140
:101E30002D933196A817B907D1F70DC09F0190E0F7
:101E40008D589F4FA2E7B0E0F90141919F014D935A
:101E5000A817B907C9F7F0938000E0937F0082E7E5
:101E600090E0602FBCDC0C5F0C3019F08FEF80939A
:101E700061000093600084E196B3987131F4815061
:101E8000D9F71092820010927C0001E0811100E0ED
:101E900080917000801739F0002319F4F89471D004
:101EA0007894009370008CE991E00197F1F70000BD
:101EB00080916600882321F40894E11CF11C02C083
:101EC000EE24FF2480FF20C080EC96E113C0F8943C
:101ED000E0916700F091680083E080935700E895F7
:101EE00007B600FCFDCF7894809167009091680060
:101EF00080549040909368008093670080916700C1
:101F000090916800009719F78091660081FF11C0D9
:101F1000A9E3B0E21197F1F700C0000080916700DB
:101F2000909168008F739070009711F01CDE01C0D3
:101F3000CBDD8091660082FD05C0B1E5EB16B3EC08
:101F4000FB06E0F0E1E2F1EA3197F1F700C00000B2
:101F5000F8941BBE15BA80916D00882311F409C056
:101F600002DE8091670090916800F7E180309F0762
:101F7000B8F310925F0210925E02C0CB109266001E
:101F800037CEFF920F931F93CF93DF93C8E0D0E03B
:101F900010E000E8F12EF00EF1BE25DC29E08433DC
:101FA00092070CF41F2D06952197A1F7212F2150A0
:101FB00021BFEC01012F10C016DC8453994097FF1C
:101FC00003C0909581959F4F8C179D0714F401B71E
:101FD000EC0181B78F5F81BF21B730E0812F90E0A6
:101FE00001968217930744F701BFDF91CF911F91AC
:0A1FF0000F91FF900895F894FFCFC1
:061FFA005AFF16FA401424
:0400000300001700E2
:00000001FF
